:020000040000FA
:100000008601850196018F289500030E83128C00CE
:100010000B1D0F28A008031DA0030B11502803106F
:10002000920D910D900D8F0D051A12179618252817
:100030005B210E08D83A031D4F280D08033A031D13
:100040004F2896149301013094005520940B4F28AB
:1000500002301306031D2F28D430991931281308B4
:10006000732091065B210F3084003E213F211F3019
:100070000E0503193D2896104F280310130D173E47
:1000800084000F088000840A100880001A30940051
:10009000930A131D4F2816159301F030A6008B10FC
:1000A0000C0E8300950E150E090026080F39031D4E
:1000B0006B282608F039803A031972281A30A607EF
:1000C000FF30A61B6828260E0F39173E8400000853
:1000D000A7008514722827188510271C851403147F
:1000E000A70CA603080082073F3466345A346D34E7
:1000F0008207A834A8348C34863481342D342034DB
:100100005034493443342D3452344434533420343D
:1001100032342E343034303420342D34FF348316CE
:100120004730810011308500F13086008312323073
:100130002B220A228B13422208228F019001910167
:100140009201A1019F017F30A000B0308B006400BC
:10015000200803199A280739031DB228A003532247
:100160009F0A9F13161DA72816117030A0041708A8
:10017000180621060319BF289616A106A728961E61
:10018000C428961242229F011908F0390319D12878
:10019000203A031910291908F839403A031920297F
:1001A000A7288F30F0212030191DD9282D301A1A98
:1001B0002A30F121191DDF281A1A05151A1E0511FA
:1001C0001A0D0639063A0319F128063A283E8B1310
:1001D00084001D0880388000840A1E0880008B1768
:1001E000A728A81FA728AA1FA728AC1FA728A813BD
:1001F000A913AA13AB13AC13AD138030F021280858
:10020000EE212908EE212A08EE212B08EE212C08E8
:10021000EE212D08EE211D08EE211E08EE21A72853
:100220001A0D3E39A300A3071F08A302A3131B083E
:10023000E1211C08E1211D08E1211E08E121A72878
:100240008930F0211D0E0F391C181038A2001E0C29
:100250000F399E1A003CA2071830A21BA2072202E7
:10026000031C220885223A30F1211E0DA2001D0D2B
:10027000A300220D230D3F398522A72816148030B4
:1002800094008D1C4A291F300E05031D4A291610A3
:100290001408800603108E0D8D0D161C55290D1D9A
:1002A0005529B9308E0601308D060310940C031CBD
:1002B0004129840A08008E018D01121F6329033031
:1002C0008D061B308E06921F692903308D068F30F4
:1002D0008E06111C6F2902308D06A7308E06F7306E
:1002E00091188E06111D782901308D06EE308E068C
:1002F000911D7E2903308D06DC308E06111E842967
:1003000002308D0601308E06911E8A2901308D063D
:10031000BB308E06111F902903308D0676308E0675
:10032000911F962903308D0655308E06101C9C298E
:1003300003308D0613308E06901CA22903308D06E3
:100340009F308E06101DA82902308D0687308E063C
:10035000B73090198E06101EB12901308D066E300F
:100360008E06901EB72902308D06DC308E060130D5
:10037000101B8E060230901B8E0604300F188E065E
:1003800008308F188E0610300F198E0620308F1906
:100390008E0640300F1A8E0680308F1A8E0601307E
:1003A0000F1B8D0602308F1B8D060800043086005F
:1003B00086140000060D8610861486100318D829AE
:1003C0000800A4002308231BEA29273CC030031C93
:1003D00068302307F021A30AA31324080023F1297E
:1003E0009615A200D62183160130860083122208BA
:1003F0000122220E012296118316F130860083120B
:100400000800F039961D083886008614861008000A
:1004100005301C2A96153030012203302B22303053
:10042000012201302B223030012201302B222030DA
:10043000012201302B22A30123087820FF3A03195F
:100440000800FF3AA2009615A21F96117F39A2005C
:10045000F121A30A1C2AA400A5016400A50B2D2AE2
:10046000A40B2C2A0800D621861586140000060845
:100470008610F039A20086140000060E86100F398F
:10048000220408000130F0214030A300F021203088
:10049000F121A30B472A2030A800A900AA00AB0035
:1004A000AC00AD0008000430F0214030A400F02181
:1004B0003322A3003F30A5007C22C030A400F021ED
:1004C0003322A5007F30F0212508F1212730A50037
:1004D0007C229030A400F0213322A500E730F021E7
:1004E0002508F1211730A5007C22A730F021230830
:1004F000F1210630F0210800A40A2408F02133225B
:10050000F121A50B7C2A64000800A201F63EA20A94
:100510000318862AFA3EA20E2207A300230E912278
:0E05200023080F39063E8318073E2A3EF129B4
:10060000A200A21B082BE03903192034220808009D
:100610008B1303308A000E238A01090022087F39D8
:1006200082076134613465346534693469346F3408
:100630006F3475347534EE3443345334E2346934F2
:1006400069346134E13465346534693469346F3454
:10065000EF347534F534EE34633473347134693403
:1006600069346134E03463342534473465346E349E
:100670009434F7344334ED3424347F345E347E34A0
:100680007634DF343134323433342B3449346E34FD
:10069000F534E4343F34FD34DF3420342034203466
:1006A00024344134413445344534493449344F3499
:1006B0004F34553455345234433453345A3444341B
:1006C0004C344134E13445344534493449344F34B1
:1006D000EF345534F5347234633473347A3464341B
:1006E0006C344134413445344534793459344F34D1
:1006F000303470346E345234433453345A34FA3410
:1007000064346134613465346534773479346F34FA
:10071000F23470346E347234633473347A34FA34AD
:02072000203483
:02400E00F53F7C
:00000001FF
